:020000041000EA
:1000000000B5324B212058609868022188439860DF
:10001000D860186158612E4B002199600221596106
:100020000121F02299502B49196001219960352056
:1000300000F044F80222904214D00621196600F024
:1000400034F8196E01211966002018661A6600F04E
:100050002CF8196E196E196E052000F02FF8012189
:100060000842F9D1002199601B49196000215960AB
:100070001A491B48016001219960EB211966A021F2
:10008000196600F012F800219960164914480160C1
:100090000121996001BC002800D000471248134993
:1000A000086003C880F30888084703B5996A0420EC
:1000B0000142FBD001200142F8D103BD02B5186610
:1000C0001866FFF7F2FF186E186E02BD00000240BE
:1000D000000000180000070000035F00212200005C
:1000E000F4000018222000A00001001008ED00E03C
:1000F00000000000000000000000000074B24E7A12
:1001000000200420F7010010C3010010C5010010F9
:10011000C1010010C1010010C1010010C101001097
:10012000C1010010C1010010C1010010C701001081
:10013000C1010010C1010010C9010010CB01001065
:10014000CD010010CD010010CD010010CD01001037
:10015000CD010010CD010010CD010010CD01001027
:10016000CD010010CD010010CD010010CD01001017
:10017000CD010010CD010010CD010010CD01001007
:10018000CD010010CD010010CD010010CD010010F7
:10019000CD010010CD010010CD010010CD010010E7
:1001A000CD010010CD010010CD010010CD010010D7
:1001B000CD010010CD010010CD010010CD010010C7
:1001C00000BE00BE00BE00BE00BE00BEEFF3058054
:1001D000103800BEF2EB88712C5D0010505D0010ED
:1001E0003402001090A31AE700201F49086006C8D7
:1001F00081F3088810471D48006800282FD10DA4FE
:100200000ECC002902D000F012F8F9E71849194A7B
:10021000002000E001C19142FCD1174988471749ED
:1002200088471749884700BEFDE701C901C29A42C5
:10023000FBD37047505D0010C00000200403002075
:10024000945F00100000042000000420945F001060
:10025000001004200010042000000000704709482E
:1002600003F052F90047000008ED00E0000000D064
:10027000080300200C07002019220010410500107F
:10028000D92100105756000006005250ABB36053FE
:10029000E05B001006005250861C0302F05B001069
:1002A000060052505422A29DF85B001005005250E7
:1002B000DE65F468945F0010F8B5C0460448054B4D
:1002C00010B5834203D0044B002B00D0984710BDDB
:1002D0000403002004030020000000000648074932
:1002E000091A8B10C90FC91810B5491003D0044B57
:1002F000002B00D0984710BD040300200403002009
:100300000000000010B5074C2378002B09D1FFF73F
:10031000D5FF054B002B02D0044800E000BF0123AD
:10032000237010BD0804002000000000504D001094
:10033000054B10B5002B03D00449054800E000BF71
:10034000FFF7CCFF10BDC046000000000C040020E9
:10035000504D001070B506000D1C081C03F0D4FFB2
:1003600084B2002C12D0200003F0A6FF011C281C30
:1003700003F079FF8721C90503F095FF03F0C4FF5F
:10038000C3B21B0224041C43346070BD0023F8E791
:1003900010B504001022002104F05EF880235B02F7
:1003A0002360F8235B0263608023DB02A360C02329
:1003B0001B03A360200010BD70B504000D00FFF703
:1003C000E7FF6A1C636809490B40ED012B431203E8
:1003D00013436360E268D200D208802189050A4392
:1003E000E260034A13406360200070BD7F00FEFF9F
:1003F000FFFFFF9F70B584B006000C0001AB02AA9E
:1004000003A900F00BFA051E04D1002C09D120002D
:1004100004B070BD019A0299039800F0C3F92C0052
:10042000F5E70248310001F073FFC046504D00105F
:10043000F0B5CE46474680B587B004000F00914620
:100440001E00284B98424AD007252900300000F0B2
:100450003DFA29000E9800F039FA012398460093DE
:1004600032003900200004F079FB434600930E9AD5
:100470003900200004F072FB494602A8FFF79CFFF8
:10048000059D194B1D400E9B9B021D430595174B67
:100490001D402E4380235B0333430593049B9B0045
:1004A0009B088022D205134304930F9902A8FFF7FB
:1004B00051FF049A0E4B1A400E4B1343049302ABA8
:1004C0004A463900200004F09BFB22684346BB40AB
:1004D0001343236007B0C0BCB946B046F0BD062543
:1004E000B3E7C04600002050FF83FFFFE0FF0FFC92
:1004F000FFFFF5C10000021010B5002B02DB026007
:10050000436010BD024B034A03483F2101F068FEDF
:10051000844D0010F84D0010A04D001010B582B0B1
:10052000040001F0A9F902000B006846FFF7E4FFA0
:10053000009A019B22606360200002B010BD0000A1
:1005400030B587B004F02AF901211848FFF752FFAF
:100550001749184C200004F0E5FA0200FE239B0521
:10056000019312230093013300212000FFF760FF65
:10057000114800F0B9F802A8FFF7D0FF029C039DD4
:10058000002000F0E7F80D4800F0E4F8002000F04B
:10059000E1F802A8FFF7C2FF029A039B121BAB41CE
:1005A00004920593064804F0EDF8E4E7400D0300DB
:1005B000344E001000002050104E0010FFFF0000CD
:1005C000F04D001070B504000D000120002101F075
:1005D000C7F80B49486901231A00824009698B401A
:1005E000134384408D402C43D022120611694C40A5
:1005F0001C40D4610120002101F0B2F870BDC0465A
:10060000DC060020F0B5D6464F464646C0B505008C
:100610000F00140099460B00183301269E40866097
:10062000AB683342FCD000210020FFF7CBFF631CF6
:100630009A4621786A683B00103301249C402300CD
:10064000134098461442F5D10437BF00EF193970B2
:100650004B46012B18D9AE60AB683342FCD0002169
:100660000120FFF7AFFF0BE05346013352461178EC
:100670006A682242FCD1397001229446E0449A46CD
:100680004B46013B4345EFD8AE60AB683342FCD0EC
:1006900001210120FFF796FFE0BCBA46B146A8460B
:1006A000F0BD70B506000D0014000AE0A21C290080
:1006B0003000FFF7A7FFC82001F05FF8237802336E
:1006C000E4182378002BF1D170BD00B583B06B46E0
:1006D000DA1D2C2313702B3BFFF794FF0021012020
:1006E000FFF770FF03B000BD70B50100174C242266
:1006F000200003F0B7FE206900F000F9606900F007
:10070000FDF8A06900F0FAF8E06900F0F7F8236955
:10071000012632009A40D0252D066A6263693100B5
:1007200099406962A369310099400B006962E169EF
:100730003000884068626A616B61054A61682068C0
:10074000FFF7AFFFE3699E406E6170BDDC060020DD
:10075000404E0010F8B50500114C61682068FFF7A5
:10076000B4FF238C678C5F43002616E00C4B1A689D
:100770005C682B0A9C46516820001030012383409E
:100780000B42F8D10434A400141961462170E8B278
:1007900051680B42FCD120700136BE42E6DBF8BD49
:1007A000DC060020F0B583B004000D00160000F058
:1007B000B1F8002801D003B0F0BD154F00973B0001
:1007C00001220121053001F04BFB00962B00220095
:1007D0000121104801F04CFC31006943200002F077
:1007E000E7FE04000C4B009300220221042001F0DC
:1007F00037FB0094230000220121052001F030FB8B
:1008000000973B0002220021062001F029FBD2E7DD
:10081000006CDC0200800240001BB700F0B5DE4631
:1008200057464E464546E0B583B080468B4600921B
:100830000193042001F016FCFA21890002F0B8FEB1
:100840008246A0235B0099462CE0013C002C20D07E
:1008500025007D432900300002F0AAFE4045F4D176
:100860002900300002F0A4FE0029EED173019B1B89
:100870009B009B19DB005A461360009B1F60019B85
:100880001C60012003B0F0BCBB46B246A946A0469E
:10089000F0BD013F002F01D03C00D7E701235B42B0
:1008A0009C46E1444B460F2B09D956464B465E43C6
:1008B000044BF218044B9A42F0D80727EAE70020CD
:1008C000E0E7C046508EF4FF50F80C0010B58300EE
:1008D000084A944663441A684024624080341440B5
:1008E0008022520113431C60C000034B9C466044AD
:1008F000416010BD04C001400040014010B501231B
:100900008340D0221206936293610521FFF7DEFF38
:1009100010BD0000034B1B6802201840431E984185
:10092000C0B2704700C00640EFF3108072B6034BB0
:100930001B68002BFBD0BFF35F8F70472C0100D0EA
:10094000BFF35F8F024B00221A6080F3108870475C
:100950002C0100D0F8B506000C001500FFF7E4FFED
:10096000E308F718F15C07222240012393400B4271
:1009700005D1DBB20B433B70FFF7E2FFF8BD21006E
:10098000280001F0C5FC0000002307E0054A9A1882
:100990009200BFF35F8F0021116001331F2BF5D947
:1009A0007047C04640000034054A1078431CDBB253
:1009B0001370172B02D9130010221A707047C0460B
:1009C00038020020074B9B68103080001950BFF39D
:1009D0005F8FBFF35F8F044B0021196082F3108893
:1009E0007047C04600ED00E0240100D010B5038838
:1009F000DA0A1C2A05D15B055B1502335B00C018BF
:100A000010BD034B034A0448B12101F0E9FBC04685
:100A1000644E0010085000107C4E001010B5091AEA
:100A20000B1F0A4A88180A4A904208D8C90706D4F8
:100A30005B105B055B0D0748184380B210BD064B89
:100A4000064A0748A32101F0CBFBC046FC07000083
:100A5000FE0F000000E0FFFFC44E0010FC4F00102E
:100A60007C4E001010B5091A04394A08090B08D148
:100A70004905490D064B0B430380064B1343438046
:100A800010BD054B054A0648AB2101F0A9FBC04645
:100A900000F0FFFF00F8FFFFF44E0010D04F0010F1
:100AA0007C4E001001238340034A10681840431E07
:100AB0009841C0B27047C04600E100E0002904D070
:100AC000034B1860034B18607047034B1860FBE73B
:100AD00080E200E000E100E080E100E010B50123E9
:100AE00083401800FFF7EAFF10BD0000024B9B682F
:100AF00010308000C058704700ED00E070B5040071
:100B00000D00EFF3108672B60C4B1B68002BFBD068
:100B1000BFF35F8F2000FFF7E9FF094B984201D038
:100B2000A84205D1320029002000FFF74BFF70BD1D
:100B3000044B054A0548862101F052FB240100D0F0
:100B4000CD010010044F0010185000107C4E001012
:100B5000F0B5CE46474680B583B006000D00EFF3F2
:100B6000108872B64F4B1B68002BFBD0BFF35F8F12
:100B70004D4B9A6834001034A300D7584B4B9F421A
:100B800007D0AF4200D18BE00197494BFB1A2F2BC6
:100B900009D9424639003000FFF714FF03B0C0BC4A
:100BA000B946B046F0BD3000FFF77CFF814600211A
:100BB0003000FFF793FFBFF35F8FEFF3058100294C
:100BC00001D08C4211D10123019C9C430020A368D9
:100BD000AB4212D00622A256002A0DDB53009B180E
:100BE0009B00334A2000D418F1E7324B324A3621B9
:100BF0003248FF3101F0F4FA2000AB4249D106251A
:100C00006557002D2BDB2A4B6A00521992009B1866
:100C10009A68A260DA79E2719B795BB2A371002BCA
:100C20000FDA2748A080224B6A00521992009B18C5
:100C3000244A11789971157049463000FFF74EFF2C
:100C4000A7E7680040198000194BC0180430FFF76F
:100C5000CDFE0100231D1800FFF7E0FEE2E70029AA
:100C600012D100280ED0FF238371174B83801549C2
:100C70000B78A3710E4A154BA41A644163431B0DF4
:100C80000B70D9E7094FF2E71149201DFFF7EAFE83
:100C9000D2E7104B084A6A210848FF3101F0A0FA58
:100CA000024F76E7240100D000ED00E0CD010010F6
:100CB0003C0200203C4F0010E84F00107C4E00101A
:100CC00001BD00000907002001BDFFFFAAAA000026
:100CD00076020020704F001070B5012202432E4BA7
:100CE000D31A2F2B28D8EFF30583002B2BD0EFF34B
:100CF000108C72B6294909680029FBD0BFF35F8FB9
:100D0000254C274905002D1B6D416943090D4CB247
:100D1000244989689B00C95891421BD000210329AE
:100D200032D81D4B4A00521892009B189B795BB237
:100D3000A3421FD00131F2E71B4B1C4AC7211C48BC
:100D4000490001F04DFA1B4B184A92211848FF3117
:100D500001F046FA134A92681749D150174B1A7896
:100D600082711C70BFF35F8F0C4B00221A608CF3F2
:100D7000108870BD084B4A005518AD005D19FF265C
:100D8000AE710F4AAA80E9E70E4B084AD121084804
:100D9000490001F025FAC0463C020020240100D0A1
:100DA000AAAA000000ED00E0784F0010B44F001038
:100DB0007C4E0010A04F0010CD010010090700204C
:100DC00001BDFFFFAC4F00100022044B02E00449BC
:100DD00002C30132072AFAD97047C04600E400E096
:100DE00080808080024B9C4661448900016070478E
:100DF0004000003410B50400FFF7D6FD01002000CC
:100E0000FFF7F0FFFF232371BFF35F8F10BD10B515
:100E10000400FFF7C9FD01002000FFF7E3FFFF23F7
:100E2000237100236371BFF35F8F10BD084B5B6AB2
:100E3000994209D8064A926A824207D2994201D061
:100E4000012002E0002000E0002070470120FCE7C4
:100E50000040054010B500290AD003681B7B8B4277
:100E600006D38068054B9C4661440901401810BDBB
:100E7000034B044A04483C2101F0B2F9FFFFFF0F85
:100E8000F05000102854001014510010F8B5040060
:100E90001700FFF7DFFF0668456839002000FFF7FD
:100EA000D9FF026843680120AB4201D802D000207C
:100EB000C0B2F8BDB242FBD8F9E7000010B5002B74
:100EC00002DB0260436010BD024B034A03483F212E
:100ED00001F086F9844D0010F4530010A04D00106D
:100EE00010B582B004000498059912184B41002BEC
:100EF00009DB6846FFF7E2FF009A019B226063600E
:100F0000200002B010BD01225242014BF1E7C04661
:100F1000FFFFFF7F10B5002908D0037B8B4205D36C
:100F200000684B005B18033BC01810BD024B034A1E
:100F30000348682101F054F958510010D0530010B3
:100F40007451001010B5437B8B4201D1012010BDBC
:100F5000FFF7E0FF8378002B01D10020F7E70120A5
:100F6000F5E770B50400857B002D01D1280070BD28
:100F70002900FFF7CFFF4378A373002B00D1E37361
:100F80000023837043700370F0E70000F8B506009B
:100F90000C001500FFF7BEFF0700002C0DD0002D40
:100FA00011D0AC4215D029003000FFF7B3FF847098
:100FB0003B78002B13D13D70F8BD0A4B0A4A0B4811
:100FC0006F2101F00DF90A4B074A0848702101F022
:100FD00007F9084B044A0548712101F001F94370F3
:100FE0003D70E9E7C8510010AC5300107451001077
:100FF000D4510010E051001070B506000D0014002F
:10100000002914D0002A14D043688068984700282B
:1010100006D0220029003000FFF7B8FF280007E0C3
:101020002A0021003000FFF7B1FF200000E010008F
:1010300070BD0800FCE7000070B504000D1E0CD068
:10104000FFF768FF0023837043700370617B2A0001
:101050002000FFF7D1FF607370BD034B034A0448C3
:10106000A52101F0BDF8C046F8510010C053001092
:101070007451001070B504000D1E0FD0FFF762FF11
:1010800000280BD1E17B00290ED1A37B002B03D1DB
:10109000E37B002B0DD1A573E57370BD084B094AA6
:1010A0000948F62101F09CF82000FFF733FF457056
:1010B000EBE7064B034A0448FB2101F091F8C046D8
:1010C000FC5100109C53001074510010205200106D
:1010D00010B5002907D003681B7B8B4203D3C0687F
:1010E0000139401810BD034B034A0448412101F067
:1010F00077F8C046F05000108853001014510010CB
:1011000070B505000C00080000F092FC09492000B1
:1011100000F0D2FBFFF748FC074B9C466044800080
:1011200068602C75D0231B061B786B75034BA400DD
:10113000E55070BD4D12001040000034B404002092
:101140000A4B1A68EFF3108172B61368002BFCD0BB
:10115000BFF35F8F054B1B68BFF35F8F00221A60E0
:1011600081F3108840BF002000217047C80600208E
:1011700010B582B0040000F07FFB02000B0068464F
:10118000FFF79CFE009A019B22606360200002B082
:1011900010BD70B584B0040016001D0002A8FFF752
:1011A000E7FF029A039B009601952000FFF798FE47
:1011B000200004B070BD0000F0B583B007000192BC
:1011C0001D000AAB1C780BAB1E78002C0BD00068FE
:1011D0002100FFF7B7FE002809D0194B194A1A4819
:1011E000672100F0FDFF0068FFF7BBFE0400002C44
:1011F00002D1200003B0F0BD21003800FFF72AFE25
:10120000019B03604560089B8360099BC36038684D
:101210002100FFF711FFA042EBD1387D019A2B008E
:1012200000F092FB051E01D0002E04D00C9B002B79
:10123000DFD01D70DDE73868210000F03FFDF5E7E5
:1012400034520010DC53001014510010F0B5DE468B
:1012500057464E464546E0B58FB00B900021784B7F
:101260008200D458894682E029002000FFF7F2FD71
:10127000804602684368921BBB41002B09DD434650
:101280001A685B680B9800F05FFB00239846002605
:1012900089E0002B01D1002AF1D10021584600F04D
:1012A00003FD0700A84215D143461A685B680892FF
:1012B000099343469E68DB689846002E10D02900AB
:1012C0002000FFF705FF037899461B021F432761A3
:1012D000002068E05B4B5C4A5C488E2100F080FF98
:1012E0005B4B594A5948922100F07AFF2369002B41
:1012F00077D0BB4219D106980799002342428B410F
:1013000000920193089A099B0CA8FFF7E9FD0C9A3B
:101310000D9B0021049101310391029541460191F9
:1013200000962000FFF748FF16E04A4B464A474820
:10133000A12100F055FF069A079B002B01D1002A3E
:1013400052D120682900FFF795FE29002000FFF701
:10135000BFFE037801330370002323616268BFF38B
:101360005F8F13608AF310880120002861D00CA8D9
:10137000FFF7FEFE0C9E0D9F0022002308920993AA
:101380006268EFF3108A72B61368002BFCD0BFF3CB
:101390005F8F23689B465D7B002D00D064E70023B0
:1013A0009846002600206368BFF35F8F00221A6012
:1013B0008AF31088002ED8D04B461F022F43414697
:1013C0003800B047069007916268EFF3108A72B652
:1013D0001368002BFCD0BFF35F8F079B002B00DA54
:1013E00084E7079B002BA6DD2369002BA9D0BB4215
:1013F00019D10CA8FFF7BCFE0C9A0D9B0698079913
:10140000009001910CA8FFF76BFD0C9A0D9B002139
:10141000049101310391029541460191009620000B
:10142000FFF7CAFE98E70B4B074A0848A42100F0D3
:10143000D7FE0FB0F0BCBB46B246A946A046F0BDF1
:10144000B40400205C5200100C5400101451001021
:10145000745200108052001010B50C4B5B68002BCA
:1014600004D00B480A21FFF7BDFC10BD074C094A08
:1014700020682300102100F082FB032000F0F0F927
:1014800003212000FFF73CFEEBE7C046840200206A
:10149000C80600208D0E001010B5064B5B68002BAF
:1014A00001D0044810BD044B044A05485E2100F0F9
:1014B00097FEC04684020020BC52001070530010FA
:1014C00014510010F0B5DE4657464E464546E0B58D
:1014D0008DB0060090461F00169B9A46179B9946B2
:1014E00018AB1B780793272302AA94466344002273
:1014F0001A7021E001003000FFF7EAFD00783CE0BF
:101500000698002B5CD0079B002B59D04946D0474A
:1015100004000D0003000B4359D0002940DB08A84C
:10152000FFF726FE089A099B0094019508A8FFF78B
:10153000D7FC089B9846099F7268EFF3108B72B630
:10154000136859424B41D9B20691002BF8D1BFF331
:101550005F8F273302AA94466344049300230393C6
:1015600002934B4601935346009342463B003000A2
:10157000FFF722FE0400051EBCD17368BFF35F8F26
:10158000002119608BF31088002D17D0272302AAA1
:10159000944663441B78002BB2D100022043B0E78D
:1015A00000236242AB410092019342463B0008A8EF
:1015B000FFF796FC089B9846099FBDE70120404233
:1015C0000DB0F0BCBB46B246A946A046F0BD069899
:1015D000F6E7F0B5C64600B584B0050088461600AB
:1015E0001F000AAB1C78FFF757FF02940197009683
:1015F0002A004346FFF766FF04B080BCB846F0BD42
:10160000F0B5C64600B504000D004268EFF3108740
:1016100072B61368002BFCD0BFF35F8FEEB2236865
:10162000984631001800FFF78DFC00282AD0236966
:10163000AB4213D02D0AEDB231002000FFF748FD78
:101640000378AB4211D000206368BFF35F8F0022A4
:101650001A6087F3108880BCB846F0BD0C4B0D4A69
:1016600095210D48490000F0BBFD3100404600F0D7
:1016700025FB0028E8D1094B064A32210648FF31F4
:1016800000F0AEFD2369AB42DED100232361DBE72E
:10169000E052001058530010145100100453001071
:1016A00010B50400FFF7F8FE2100FFF7A9FF10BDF9
:1016B00030B587B004000D00EFF30583002B20D177
:1016C00006225242D31712196B418B4202D803D122
:1016D000824201D90022002304A8FFF7EFFB02A8F1
:1016E000FFF746FD02980399049A059B121A8B4155
:1016F000002B0BDC08D02000290000F0C9F807B04F
:1017000030BD144800F004FE002AF4D0124A0498B8
:10171000059900230093FFF75CFF002813DAEAE73E
:101720000E4B1A68EFF3108172B61368002BFCD0D1
:10173000BFF35F8F094B1B68BFF35F8F00221A60F6
:1017400081F3108820BF04980599FFF76FFB0028EC
:10175000E6D0D0E70853001041110010C806002061
:1017600000B583B002000B006846FFF712FD009839
:101770000199FFF79DFF03B000BD10B5FA2292005A
:101780000023002102F052FDFFF7EAFF10BD000028
:1017900030B583B005000C00EFF30583002B0FD1AB
:1017A0000B4A00230093FFF714FF00280BDD20BF36
:1017B000FFF776FF28002100FFF738FB03B030BDAC
:1017C000FFF734FBFAE728002100FFF72FFBF5E7CE
:1017D0004111001070B5EFF305801038EFF3108C55
:1017E00072B6194B1B68002BFBD0BFF35F8F012231
:1017F0001300834015494B6315490B60154909785F
:101800000C00C440224213D0104A546A124A850088
:10181000AA58944205D3114AAA580E4C99432170F4
:1018200007E00A4A031D9B0099589950002200E0E6
:101830000022BFF35F8F044B002119608CF31088E6
:10184000002A00D0904770BD280100D0004005401C
:101850003C7005400A070020CC0600202C04002024
:1018600010B50100024A034B1800FFF773F810BDD2
:101870003454001008070020044B5B6A034A906A46
:101880001900536A9942F9D17047C046004005409B
:10189000084B5B6A01E0074B5B6A8B42FBD301E0BC
:1018A000044B5B6A8B4203D1024B9B6A8342F7D3A2
:1018B0007047C0460040054070B504000E00EFF3CD
:1018C000108572B61B4B1B68002BFBD0BFF35F8FDC
:1018D000002E1CD02000FFF709F9174B83420BD0D4
:1018E00019002000FFF70AF901212000FFF7F6F8A0
:1018F0000123A340114A1360114BA400E650BFF32B
:101900005F8F0C4B00221A6085F3108870BD0C4B62
:10191000A2000021D1500122A2400A490B78934332
:101920000B7005492000FFF713F900212000FFF795
:10193000D5F8E4E7280100D0D5170010386005403D
:101940002C0400200A070020F0B5DE4600B584B064
:101950000400150001921E000293FFF78DFF03950E
:101960008E4202D84ED185424CD9EFF3108B72B61D
:10197000274B1B68002BFBD0BFF35F8F254A1778DE
:101980000125A540EBB23B431370234B5D63221D41
:1019900092000199D150214AA100029888501B6AF7
:1019A0002B4212D11C4B1B6C2B4208D00020BFF3E2
:1019B0005F8F174B00221A608BF3108823E0184BBF
:1019C000184A1948C52100F00BFCFFF755FF8E425D
:1019D00014D802D1039B834210D80E4B1B78BB4214
:1019E0000ED00D4B1D625D631F22224001239340E8
:1019F0000E4A1360074B1F700120D8E70020D6E77E
:101A00000120D4E7012004B080BCBB46F0BDC04635
:101A1000280100D00A07002000400540CC06002025
:101A200058540010C85400107C54001080E200E0AC
:101A3000EFF3108C72B60B4B1B68002BFBD0BFF37F
:101A40005F8F01238340084A136208490A789A434A
:101A50000A70BFF35F8F034B00221A608CF310886B
:101A60007047C046280100D0004005400A0700200A
:101A700010B5002908D0037B8B4205D300684B00CA
:101A80005B18033BC01810BD024B034A0348682192
:101A900000F0A6FB58510010DC55001074510010E6
:101AA000F8B506000C001500FFF7E2FF0700002C58
:101AB0000DD0002D11D0AC4215D029003000FFF719
:101AC000D7FF84703B78002B13D13D70F8BD0A4BD3
:101AD0000A4A0B486F2100F083FB0A4B074A08486B
:101AE000702100F07DFB084B044A0548712100F08D
:101AF00077FB43703D70E9E7C8510010C8550010EE
:101B000074510010D4510010E051001070B506005F
:101B10000D001400002914D0002A14D043688068F6
:101B20009847002806D0220029003000FFF7B8FFB0
:101B3000280007E02A0021003000FFF7B1FF200055
:101B400000E0100070BD0800FCE770B50500002340
:101B5000437301338373037BC373012406E02100C5
:101B60002800FFF785FF0134E4B24470297BA142CD
:101B7000F5D82800FFF77CFF0023437070BD10B537
:101B8000017342608360FFF7E0FF10BDF0B5C64609
:101B900000B505000C1E03D1200080BCB846F0BD86
:101BA000FFF766FF4678002EF6D031002800FFF7D9
:101BB0005FFF477800239846437021002800FFF715
:101BC00057FF43464370320021002800FFF79EFF75
:101BD000040039002800FFF7D9FF02002100280087
:101BE000FFF794FF0400D7E7F0B5C64600B5040040
:101BF0000D001700002927D0FFF73AFF4378002B8C
:101C000028D18378002B2BD101782000FFF7BEFF6D
:101C100006008046002F0AD0E17B002926D1A37B55
:101C2000002B03D1E37B002B25D1A573E57343463D
:101C3000002B26D129002000FFF71AFF0023437054
:101C4000300080BCB846F0BD114B124A1248382112
:101C500000F0C6FA114B0F4A0F483A2100F0C0FAC3
:101C60000F4B0C4A0C483B2100F0BAFA2000FFF75A
:101C7000FFFE4570D3E70B4B064A0748422100F0B0
:101C8000AFFA31002000FFF7F3FE00238370D1E7A5
:101C9000E4540010B4550010EC54001030550010FE
:101CA000585500102052001070B504000A00457B02
:101CB0002900FFF799FF6073280070BD70B506001A
:101CC0000C1E40D0437B8B4207D0FFF7D1FE0500AE
:101CD0008178002906D1002036E00121FFF7E4FFDA
:101CE000012031E03000FFF7C3FE0178A1420DD0A2
:101CF0003000FFF7BDFE4178A1420AD00029F7D19C
:101D0000124B134A13486B3100F06AFA6B78037078
:101D100001E06B7843700023AB706B7001222100EF
:101D20003000FFF761FF0200717B814205D0300077
:101D3000FFF7ECFE7073012006E0074B044A0548EC
:101D4000712100F04DFA002070BDC046AC4F00106C
:101D50009C550010EC5400107C55001070B5040028
:101D60000D00062000F07EF9C000290001F020FCE3
:101D7000C60908D00E4B9E4217D87F23034001337B
:101D800035005E0800E001256562A6622C348023E0
:101D90009B01234300221A60062000F063F98000B3
:101DA000A901891901F004FC70BD0026014DEBE783
:101DB000FEFF0000FFFF0000002909D00A22064BA9
:101DC0009C46604443425841044B4000C252704715
:101DD00080225200F3E7C0460080FCBF00070020CD
:101DE00070B505000C00062000F03CF9002829D051
:101DF000164B9D4227D08022D203154B1A60154BFB
:101E00001A60154B9B6811009943FAD100212800F4
:101E1000FFF7D2FF21002800FFF7A0FF29002C3197
:101E2000EB6A602253400E321A4080235B010B4361
:101E30001A600A4B2B6380239B010B4310221A600C
:101E40000323AB6470BD80221204D6E700800340F8
:101E500000E0004000F0004000C00040010300002E
:101E6000F8B5DE4657464E464546E0B506000F003B
:101E700015000A9A93424ED31A0E92461B029846B8
:101E80000A9A00234046514601F0D0FB8146740077
:101E9000A419A4002E4B9C4664446368834200D27C
:101EA0006060331FDBB29B46012B3AD9C0239B01F4
:101EB0002343802212011A60264BB200D158002918
:101EC00005D0586901F074FB01300138FDD16D0176
:101ED00023685D40E0222A4080235B0123431A608F
:101EE0005A46012A28D980239B01234380221201CC
:101EF0001A604B4663604A4600234046514601F053
:101F000095FB144BB60098510120F0BCBB46B2467D
:101F1000A946A046F8BD104B104A11482D2100F0EB
:101F20005FF9012FC2D1C0239B01234303221A6012
:101F3000A368DB07FCD5CAE72168794003220A4081
:101F40001A60A3680125BD401D42FAD0CBE7C04608
:101F50000080004044040020E85500104C5600105A
:101F6000FC55001030B583B00C2000F017F9FEF7D7
:101F7000D1FC00280DD0002304E02E4A99002E4801
:101F800088500133092BF8D92A4B2C4A5A6203B0E6
:101F900030BD2B4B00229A6700F008F9294B012233
:101FA0001A60274B5B6C012BFBD1274B03221A6075
:101FB000234B9B6B012BFBD1013300930433234A4A
:101FC0000121234800F054F805230093214A012100
:101FD000214800F04DF8214B0093002202210420FB
:101FE000FFF73EFF1E4D00952B000022012105202A
:101FF000FFF736FF104C0094230000220021072039
:10200000FFF72EFF00942300002200210820FFF795
:1020100027FF0A4B00932300002200210920FFF72D
:102020001FFF00952B00002200210620FFF718FF5C
:10203000ADE7C04644040020006CDC021BB7000082
:10204000008000403CB0004030B00040002F685994
:1020500000800240008C864700C00240001BB70091
:1020600040597307014B8000C0587047440400205A
:10207000F0B5C64600B504000D00170098460C20C8
:1020800001F096FA0600394BFA18394B9A4241D8BA
:1020900043011B1A9901C91AC9000918890138009E
:1020A00001F086FA0200103A98235B009A4237D872
:1020B0004346013B062B39D8069B013B062B35D8FE
:1020C0003F09B74238D343461E04069B1B031E43F9
:1020D0002368002B36DB274B9C4244D080235B01D6
:1020E000254A1360254A1360254A926819009143D6
:1020F000FAD12560A060221DC0239B011343212239
:102100001A602268002AFCDAE66008221A6080BCA5
:10211000B846F0BD1B4B1C4A1C48112100F060F86A
:102120001B4B194A1948192100F05AF8194B164A45
:1021300016481C2100F054F8174B134A134823216A
:1021400000F04EF822683F231340AB42C3D1A3688E
:102150001B051B0D8342BED1E368EE22D202134061
:10216000B342B8D1D3E780239B01B9E780E84BD3D2
:1021700080F8A93200C0024000E0004000F00040BA
:1021800000C000405C56001088570010BC5600107C
:1021900004570010205700106C57001080239B003C
:1021A0000343014AD362704700800540064BAA22D0
:1021B00012011A602F22DA60044B054A1A60024BA2
:1021C0005B68002BFBDA7047004002400060024071
:1021D00000B0FA0000BEFDE710B5FFF7FBFF0000FE
:1021E00030B583B00D001900002A0BD0074B084C06
:1021F000019200932B000200200002F0C3FA01209C
:10220000FFF7E8FF034B1A00F1E7C04694570010B0
:10221000A4570010A057001070B52B4B2B4A1A6022
:102220002B4B2C4A1A602C4B9A682A4B9343FAD1B9
:102230002A4C01E008CC9847294B9C42FAD3FFF77F
:1022400091FE234B274A1A60234B9B68DB43DB013B
:10225000FAD1254B40229A675A671A67DA66234CEF
:1022600009E0234B234A24488621FFF7B9FF2000C9
:10227000FEF7C0FD0834214B9C4209D22368002B95
:10228000F5D0012BEDD12000FEF7C1FD0834F2E7B7
:102290001B4DA9681B4CC022200002F0E3F8AC6083
:1022A000EFF30583002B00D000BEFEF76DFBFEF7B9
:1022B0008BFDFFF7D1F8144C01E008CC9847134B85
:1022C0009C42FAD370BDC04600E00040BFCDFBFE8B
:1022D00000F00040FE7F3C0000C00040F002002003
:1022E00000030020FFFFFF0100F00140E802002092
:1022F000D457001054580010F4570010F00200207A
:1023000000ED00E000000020000300200403002096
:102310000FB400B583B0084802F004FA049B002B08
:1023200007D005A90191180002F00CFA034802F049
:10233000F9F90120FFF74EFF4058001050580010E7
:10234000704710B5002802D00B684968984710BD47
:102350000100002007E083001B185B00501C086090
:102360001078C01830380A681378303BDBB2092B7C
:10237000F1D97047F0B5DE4657464E464546E0B5C2
:1023800083B093461F000C9B9A460D9C0E9B99466A
:102390000F9B9B0703D0B8460F00060022E0019276
:1023A000A34688464E46B9460700B44207D2551C9C
:1023B0004B4641462020B84701342A00F5E73D004E
:1023C0004F465C46019B9B46B1464646B8463700A1
:1023D0002E0007E0013C551C5346185D434639006A
:1023E000B0472A00002CF5D135003E0047460F9B30
:1023F0009B0707D4100003B0F0BCBB46B246A94609
:10240000A046F0BDB0464E46B9462F005D46531B70
:10241000B342EFD2541C4B4641462020B84722001D
:10242000F5E7F0B5CE46474680B585B09446984668
:102430000C9D0D9C0EAB1B789946109A119B129E19
:10244000B7071CD4002B0CD0F7070AD54F46002F36
:1024500002D10C37374204D0013B02E030272F5520
:102460000134944201D21F2CF8D9F70707D59C42BA
:1024700005D21F2C03D830272F550134F5E7F70676
:1024800012D5770505D4002C03D0944221D09C426C
:102490001FD00F9A102A32D00F9A022A37D01F2C41
:1024A0000AD830222A5501341F2C05D84A46002A62
:1024B00033D02D222A5501340396029301940095BE
:1024C00043466246FFF756FF05B0C0BCB946B0466A
:1024D000F0BD621E012C10D00F9F102F0BD01400E6
:1024E0000F9A102AD8D1B206D6D51F2CD4D858228C
:1024F0002A550134D3E7023CCBE71400C9E7B20602
:10250000EED41F2CECD878222A550134C7E71F2CB3
:10251000D2D860322A550134C1E7720703D52B2285
:102520002A550134C8E73207C6D520222A5501347E
:10253000C2E7F0B5DE4657464E464546E0B593B095
:1025400081468A46089209931CAB10CB1B789B46A8
:102550001E9D219B9846002C03D1102342469A438E
:1025600090468023DB0046461E4042461A4212D067
:10257000002C22D000260EE03033D9B2771C0AABF3
:1025800099552900200001F013F8AC4216D31F2FF3
:1025900014D83E0004002900200001F009F8CBB255
:1025A000092BE9D94246920605D54121C918C9B27D
:1025B0000A39C9B2E2E76121F8E7270043460693EA
:1025C000209B05931F9B049303955B460293019701
:1025D0000AAB0093099B089A51464846FFF721FF32
:1025E00013B0F0BCBB46B246A946A046F0BDF0B55C
:1025F000DE4657464E464546E0B597B00A900B91E9
:102600000C929A46209B9946219F22AA13789B46BA
:10261000249B0993259C289B98464A463A4302D11D
:102620001032934398468022D200454615404346D7
:1026300013420AD04A463A4341D000252E00534661
:102640000D934D46099B9A461BE02E0053460D9371
:102650004D46099B9A4614E03033DAB2731C994612
:102660000EAB9A55524623002800390000F0DEFFD9
:10267000BC4226D819D04B461F2B1CD84E4605000D
:102680000F00524623002800390000F0CFFFD3B2DC
:10269000092BE1D94246920605D54122D218D2B281
:1026A0000A3AD2B2DAE76122F8E7AA45E3D94E4600
:1026B0000D9B9A4608E04E460D9B9A4604E0002684
:1026C00002E04E460D9B9A4643460693279B059390
:1026D000269B0493099B03935B46029301960EABE2
:1026E000009353460C9A0B990A98FFF79AFE17B07D
:1026F000F0BCBB46B246A946A046F0BDF0B5DE46EA
:1027000057464E464546E0B591B0804689460C9204
:102710009A461A9C1B9D22002B002000290001F0E4
:1027200010FA002800D0ECE001225242D44B2000E5
:10273000290001F001FA002800D0E2E00122524213
:10274000D04B2000290001F0E1F9002800D0D8E0AA
:10275000002200232000290001F0D8F9002800D031
:10276000E4E0069407958023DB001E9A1A400D9240
:102770001E9A1A4201D106231C930698079902005B
:102780000B000892099303000A00024300D1D9E02C
:10279000080D4005400DBC4EB44660440A03120BC0
:1027A0001E00BA4B13431F0001F0DEF9B84AB94BC3
:1027B00001F069F9B84AB94B01F03EF90890099166
:1027C0000022B74B3000390001F02DF9B54AB64B65
:1027D00001F059F902000B000898099901F02CF951
:1027E00001F0DAF9834601F0BFF906000F00AF4AA5
:1027F000AF4B01F048F90022AE4B01F01DF901F09A
:10280000CBF90890AC4AAD4B3000390001F03BF9F0
:1028100006000F00089801F0A7F9A94AA94B01F09A
:1028200032F902000B003000390001F0FCF806001C
:102830000F0002000B0001F026F90A900B91089B93
:10284000A14A9446634400210022089109921B0585
:1028500009930023089332003B003000390001F057
:10286000EBF80E900F9132003B0000208021C9054B
:1028700001F0D9F806000F000022944B0A980B993A
:1028800001F0E3F80022924B01F0D6F802000B00B1
:102890000A980B9901F0D9F800228E4B01F0CCF880
:1028A00002000B000A980B9901F0CFF802000B0010
:1028B0003000390001F0C0F802000B000E980F99AB
:1028C00001F0C3F80022714B01F0B6F8089A099B99
:1028D00001F0D9F806000F0008960997069A079BA1
:1028E00001F02AF900282FD001235B429C46E344E3
:1028F0000022774B3000390001F0A7F808900991C9
:1029000022E01E9B04931D9B03931C9B0293009447
:10291000019553460C9A4946404600F0FFF811B025
:10292000F0BCBB46B246A946A046F0BD002100223D
:1029300006910792069480231B069C46AC4463468E
:10294000079310E700239B465B466333C62B20D8D2
:1029500004261E9B1B0528D5089A099B19001143C4
:102960000FD05D4A5D4B0698079901F0DDF800280D
:102970007AD000225A4B0698079901F0C7F8002830
:1029800072D01C9B5B4506DD5A469B1A013B1C938B
:1029900003E00526DDE700231C938023DB001E9A5D
:1029A0001A431E92002600239B461D9B9E4265D221
:1029B0009F1B02231E9A1A400A921E9A134202D0AB
:1029C000002E00D000275B46002B07D0089A099BF9
:1029D0000698079901F039F8069007910022002324
:1029E0002000290001F092F8002800D07CE03D4B47
:1029F0001E9A1340049303971C9B0293069B079C0B
:102A00000093019453460C9A4946404600F086F8DC
:102A1000002E00D183E71E9B9B0671D54525441CE3
:102A20005346020049462800C0475A46D317D218D9
:102A30005A4005230593013E0496002303930A336D
:102A400002935B46DB0F01930092534622004946F6
:102A50004046FFF76EFD0A9B002B00D15FE70200A6
:102A600047460C9E1D9D53E01C9B002B9DD00D9B4B
:102A7000002B9AD01C9B013B1C9396E7002798E7FC
:102A8000FFFFEF7FFFFFEFFF01FCFFFF0000F03FC4
:102A9000FB799F501344D33FB3C8608B288AC63F4D
:102AA0000000F83F61436F63A787D23F71A37909A4
:102AB0004F930A400000E03F1655B5BBB16B024092
:102AC000EF39FAFE422EE63FFF03000000002C40E3
:102AD00000002440000018402D431CEBE2361A3F52
:102AE00080842E41FFF7FFFF069C079D22002900EE
:102AF00080200006844661440B000692079376E727
:102B000065258CE7541C534649462020B8472200CF
:102B1000931BAB42F6D3100001E7C046F0B5DE468A
:102B200057464E464546E0B595B006900791934608
:102B30009946209F1E9A1F9B1000190001F001F872
:102B4000002831D101225242BF4B1E981F9900F03C
:102B5000DDFF002837D101225242BC4B1E981F993D
:102B600000F0EAFF00283DD10022B94B1E981F99C2
:102B700000F0E2FF002850D10022B64B1E981F99AA
:102B800000F0C4FF002848D1002200231E981F999E
:102B900000F0BCFF002850D100239846229B5B0523
:102BA00000D4B6E0002458E0229B0393219B0293BB
:102BB00003230193A84B00934B465A460799069866
:102BC000FFF7D8FB0EE1229B0393219B0293042382
:102BD0000193A24B00934B465A4607990698FFF77C
:102BE000C9FBFFE00423229A1A4022990B4210D01D
:102BF0009B4B002A0FD00422229903912199029124
:102C0000019200934B465A4607990698FFF7B2FB8C
:102C1000E8E0944BEDE70322EEE7229B0493219B2F
:102C2000039302971E9B1F9C009301944B465A46A8
:102C300007990698FFF762FDD4E01E9A1F9B0020BB
:102C4000002100F0F0FE1E901F9101239846A5E799
:102C50000CAB30221A55013F01341F2C01D8092F2B
:102C6000F6D81E981F9900F097FF050000F07CFF32
:102C700002000B001E981F9900F0D5FE7A4BFA0057
:102C80009B181A685B680A920B9300F0FCFE089090
:102C9000099100F0A5FF060000F062FF02000B00A2
:102CA0000898099900F0BFFE0890099100226F4B27
:102CB00000F042FF00282ED00136300000F050FF17
:102CC00002000B000A980B9900F026FF002801D0A3
:102CD00001350026002F2CD1280000F045FF02000E
:102CE0000B001E981F9900F09EFE06000F000022A8
:102CF0005E4B00F00BFF002846D100225B4B3000FA
:102D0000390000F019FF00283ED1EB073CD5013512
:102D10003AE0062746E70022544B0898099900F04C
:102D2000F5FE0028D6D1002E01D0F307D2D501360A
:102D3000D0E7AA461F2C11D8013F0A21300000F02D
:102D400037FC651C30310CAB19550A21300000F0FE
:102D50002FFC092E0ED906002C00EBE755461F2C40
:102D60000CD87B1E002F09D00CAA302111551F0052
:102D70000134F4E72B0055461C00F0E71F2C03D864
:102D80000CAB2E221A5501341F2C10D80A21280012
:102D900000F0E6FB661C30310CAB19550A21280007
:102DA00000F0DEFB051E01D03400EDE73400032304
:102DB000229A1340012B1CD01F2C06D84346002B0F
:102DC00032D00CAB2D221A550134229B0393219B48
:102DD000029301940CAB00934B465A460799069810
:102DE000FFF7C8FA15B0F0BCBB46B246A946A046EC
:102DF000F0BD219B002B13D04346002B02D10C3396
:102E000013420FD0219B013B2193190003E00CAB2F
:102E100030221A5501348C42CED21F2CF7D9CBE781
:102E20002199F8E72199F6E7229B5B0704D50CABC3
:102E30002B221A550134C8E7229B1B07C5D50CABC2
:102E400020221A550134C0E7FFFFEFFFFFFFEF7F9D
:102E500065CDCD4165CDCDC17058001074580010BE
:102E6000645800106C580010185A00100000E03F21
:102E7000F0B5DE4657464E464546E0B593B082462D
:102E8000884693461193002900D10DE3002556464C
:102E9000119B1878002800D109E3252809D06C1C63
:102EA0005B462A004146B047119B01331193250030
:102EB000EEE701331193002720E001231F43013285
:102EC0001192012418E002231F43013211920124C0
:102ED00012E004231F430132119201240CE0082365
:102EE0001F4301321192012406E010231F430132D7
:102EF0001192012400E00024002C09D0119A1378CB
:102F0000203BD9B21029F6D88B00C849CB589F4630
:102F1000119B1A781300303BDBB2092B10D92A2AF7
:102F200013D00B94119B1A782E2A1ED0119A137865
:102F3000683BD9B2122959D88B00BD49CB589F465E
:102F400011A8FFF705FA0B90ECE71C9B1A1D1C92C9
:102F50001B68002B04DB0B93119B01331193E1E7FA
:102F6000022217435B420B93F6E78022D2001743FD
:102F70005A1C11925A781300303BDBB2092B0BD943
:102F80002A2AD3D11C9B1A1D1C921C68002C08DB1A
:102F9000119B01331193C9E711A8FFF7D9F9040078
:102FA000C4E70024F4E780235B003B43511C1191EC
:102FB00051786C2901D01F0018E0C0239B001F43EB
:102FC0000232119212E080233B43511C119151783F
:102FD000682901D01F0009E0C0231F43023211926B
:102FE00004E080235B001F4301321192119B18788B
:102FF000672818D8252800D24CE20300253BDAB216
:10300000422A00D946E293008A4AD3589F46802339
:103010009B001F4301321192E8E780235B001F43AE
:1030200001321192E2E7782800D933E2692800D210
:1030300030E20200693AD2B2012393407E4A134241
:1030400011D11A0600D500E25B0500D422E21C9BD8
:103050001A1D1C921B689A46002C00D0B2E1012276
:10306000524253468EE16F280ED006D858283DD0E4
:10307000622804D102239C4608E0782839D0102326
:103080009F43063B9C4601E008239C46582833D0CA
:10309000692803D0642801D00C2297437A0501D512
:1030A0000122974369282AD0642828D0BA0500D580
:1030B0009FE0FA0500D5C1E07A0600D4D3E01C9A5F
:1030C000111D1C911168FF220A4005970B9B049368
:1030D0000394634602930023019300925B462A0007
:1030E00041463000FFF725FA050027E010239C46F3
:1030F000CCE710239C46C9E720221743C8E7BA054E
:1031000020D4FA0550D47A0666D51C9A111D1C915C
:103110001168FF220A40D0171118414005970B9BF8
:103120000493039463460293D20F019200915B468D
:103130002A0041463000FFF7FCF90500119B0133DE
:103140001193A5E61C9A073207218A431100083122
:103150001C91116853689946DB170C930D930C9AD8
:103160000D9B100048400E904A4653400F930E9816
:103170000F990C9A0D9B801A99410E900F91089708
:103180000B9B0793069463460493002305934B46D9
:10319000DA0F0292009001915B462A00414630000E
:1031A000FFF725FA0500C9E71C9A111D1C9112684A
:1031B000D0171118414005970B9B04930394634665
:1031C0000293D20F019200915B462A0041463000E3
:1031D000FFF7AFF90500B1E73A0605D51C9A111DB6
:1031E0001C910023D25E96E71C9A111D1C91126857
:1031F00091E71C9A073207218A43110008311C917C
:1032000008970B9B0793069463460493002305934A
:10321000029353681268009201935B462A0041466C
:103220003000FFF7E4F9050088E7C0467C5800103D
:10323000C05800100C590010419000001C9A111D3C
:103240001C9105970B9B0493039463460293002300
:103250000193136800935B462A0041463000FFF754
:1032600068F905006AE73A0606D51C9A111D1C91FB
:1032700012681204120C28E71C9A111D1C91126886
:1032800023E7462819D01C9B0733072293431A00D3
:1032900008321C9204970B9A039202941A685B6896
:1032A000009201935B462A0041463000FFF736FC4E
:1032B0000500119B01331193EAE520231F43E2E748
:1032C000672801D0472802D180231B011F434528CE
:1032D00001D0472801D120231F431C9B073307221D
:1032E00093431A0008321C9204970B9A039202949B
:1032F0001A685B68009201935B462A0041463000E1
:10330000FFF7FCF90500119B01331193C0E502237F
:103310001A003A4091463B421DD001241C9B1A1DC5
:103320001C926F1C18785B462A004146B0474B46FA
:10333000002B14D1119B013311933D00A8E5571CBC
:103340005B4641462020B04723003A005C1C9D426A
:10335000F5D81500E2E701232A000B9DF6E73A00B5
:10336000B1460B9E06E0571C5B4641462020C847ED
:103370002C003A00651CA642F5D817004E46D9E746
:1033800001330A001978002902D0511E002AF7D112
:1033900052469B1A8022D2003900114089461742BA
:1033A00002D0A34200D9230002221100394010911B
:1033B0003A4209D02A00250057469A4633004E4625
:1033C000994621E022004CE62A004546A04606E048
:1033D000541C5B4629002020B0473B0022005F1CA4
:1033E0000B999942F4D84446A8463B00250057461D
:1033F0009A4633004E46994606E01D000137541C9C
:103400005B464146C84722003878002804D0002E89
:10341000F4D06B1E002DF0D1150053464E46109A85
:10342000002A03D1119B0133119331E50B9F2A0030
:1034300006E0551C5B4641462020B04723002A0089
:103440005C1C9F42F5D81500ECE721233B431C9AF6
:10345000111D1C91126805930823049303940833EB
:1034600002930023019300925B462A0041463000FC
:10347000FFF75FF80500119B0133119308E56C1C01
:103480005B462A0041462520B047119B013311932A
:103490002500FDE46C1C5B462A004146B047119BA9
:1034A000013311932500F3E40A4B9A46EEE4B24649
:1034B0005D450DD35B465A1E5B4641460020D04712
:1034C000280013B0F0BCBB46B246A946A046F0BDEA
:1034D0002A00F1E74123001000B585B00290039166
:1034E00001210448009313004A4202A9FFF7C0FCDF
:1034F00005B000BD4323001001480421014B1847CB
:10350000B00200202935001010B5010018231B88D7
:1035100014221088984710BD10B5010018231B888D
:1035200016221088984710BDF0B5C64600B50700B2
:103530000E0000250123984600E00135B5420AD26D
:10354000AC003C192068FFF7DFFF20600028F4D1B1
:1035500000239846F1E7404680BCB846F0BD000025
:10356000124A936F9B0815D29066D166002905D048
:10357000FFE7FFE7FFE7516F106F704704B5802149
:103580000906C2175140002800D0C84301F0D0FB03
:10359000002104BDF0B5146E556E576F166FFFF71E
:1035A000E3FF1466556657671667F0BD000000D04C
:1035B000114A936F9B0813D210665166002905D0FB
:1035C000FFE7FFE7FFE7516F106F704704B5002872
:1035D00001D00020C04301F0ABFB002104BDC04678
:1035E000F0B5146E556E576F166FFFF7E5FF146652
:1035F000556657671667F0BD000000D094464A4AEA
:10360000926F9208624601D228E0C046F0B5464E5D
:10361000346E756E776F366F00F020F89446424A2C
:1036200014665566576716676246F0BD94463E4A73
:10363000926F9208624601D254E0C046F0B53A4E0D
:10364000346E756E776F366F00F04CF89446364ADC
:1036500014665566576716676246F0BD002B24DB7B
:1036600011D000293EDA00B5C943404200D10131F2
:1036700000F038F8C943404200D10131DB435242E7
:1036800000D1013300BD002AEBD1002801D100296F
:1036900005D00020C90FC90701D1C043410800B5BA
:1036A00001F03EFB0022002300BD00B500290ADB2B
:1036B000DB43524200D1013300F014F8C9434042C9
:1036C00000D1013100BDC943404200D10131DB438B
:1036D000524200D1013300F005F8DB43524200D1E1
:1036E000013300BD002923D1002B18D1002A0CD0B2
:1036F000BC460D4F38667A6600210023FFE7FFE7DE
:10370000FFE77A6F386F67467047002801D0074897
:10371000010000B501F004FB0022002300BD0200FF
:103720000B00002000217047000000D0FFFFFFFFCA
:10373000002B00D0BFE0130C28D1002AE7D080B4C2
:10374000114F39667A66FFE7FFE730B4040C7B6FF0
:10375000396F1B0423433B667A66FFE7FFE7FFE709
:10376000C04684B27B6F3D6F1B0423433B667A6681
:10377000FFE7FFE7C04600232C042D0C7A6F386F5B
:1037800000196941B0BC7047000000D0F0B5944604
:103790000025140E01D112020835140F01D11201B7
:1037A0000435940F01D192000235D40F01D152009B
:1037B0000135D40B0134254F7C66254C3C660E0C3C
:1037C00093B2FFE7FFE7FFE73C6F6643360C7703F2
:1037D000BE467343DF0B5B04C01AB941130C73433D
:1037E000DB18C91ACE086643360CB64493B273434D
:1037F0001F0F1B01C01AB941130C73431F0B1B058C
:10380000C01AB941860D8F023E436643360C092D1E
:1038100024DB520A7243801A7703460A6643360C49
:1038200016235B1BDE40DF40BF1964466643821BE4
:103830007046043506330100D940A840C01900D3B2
:103840000131A24206D20023F0BD0000000000D0EA
:10385000FFFFFFFF121B0130F3D3F1E709277F1BA6
:10386000FE406446A2B27243801A00D20139220C93
:103870007243130C1204821A99410B0070460435EE
:1038800013370100F940A840801900D30131002B03
:1038900002D1A2420AD2F0BD013000D30131121B85
:1038A000FAD2013BF8D1A24200D2F0BD013000D3E0
:1038B0000131121BF7E7F0B51C0C00D080E00CB40E
:1038C00000251C0A04D11B02160E334312020835D0
:1038D0001C0B04D11B01160F3343120104359C0B42
:1038E00004D19B00960F334392000235DC0B02D1CA
:1038F00092185B4101351C00971864410134464F12
:103900007C66464C3C660E0CFFE7FFE7FFE7C046CF
:103910003C6F6643360C7703BE4697B27743C01BB5
:1039200000D20139C01B00D201399FB27743C91BB5
:10393000C91B170C77437E04FF0B801BB941CE08CF
:103940006643360C0C2D33DBB644120B1F053A438D
:103950001B0B97B27743C01B00D201399FB277434C
:10396000C91B170C77433E043F0C801BB941860DE1
:103970008F023E43664329277F1BFE400C3D77465E
:10398000AF40BF1930BCA2B2ABB272437343801ACE
:103990009941220C7243130C1204801A99410200BF
:1039A0000B000137001BA941F9D2781E0021F0BDA0
:1039B0000C277F1BFE4077467F0BAF40FF19E0E7E7
:1039C00000245D1C07D0144F7D663966FFE7FFE7D2
:1039D000FFE7FFE73C6F95B29EB265436643401B2D
:1039E000B141150C1E0C6543664336042F0C3E4353
:1039F0002D04401BB141994204D202000B0020006B
:103A00000021F0BD01D19042F7D3801A99410134D1
:103A10009942F2D3F6E70000000000D0FFFFFFFF5D
:103A200048404140484018B41B4B5B68FC4601933A
:103A300008BD04DFFF3C001018B4174B1B68FC46A0
:103A4000019308BD00DF093D00109446134A926FB0
:103A5000920809D2624618B40F4BDB68FC4601930A
:103A600008BD0CDFC13F00100C4AF0B5146E556E56
:103A7000576F166F6246FFF7EEFF084A14665566E9
:103A800057671667F0BD18B4034B9B68FC4601935B
:103A900008BD08DF653E0010C4040020000000D00F
:103AA000FFB550404240504059404B40594000E023
:103AB000FFB5154F4C00640D03D0BC4204D10C037C
:103AC00014D80020090D09055C00640D03D0BC4228
:103AD00004D11C030AD800221B0D1B0501264B40F4
:103AE00009D44B4003D58B4200D18242FFBD99429D
:103AF000FCD19042FFBD0B43DB1803431343F5D0C9
:103B0000C9434918FFBD0000FF07000000B5FFF7DB
:103B1000CFFF804100BDC04600B5FFF7C9FF01D906
:103B2000002000BD012000BD00B5FFF7B9FF01D99D
:103B3000002000BD012000BD00B5FFF7B1FF8041AE
:103B400000BD012040054A00121804D85A0012187E
:103B500001D8002070470120704700207047000006
:103B60000021002805D17047C1174840401AFAD0FB
:103B7000C90713B5064B1B6898470CBC441CA240F0
:103B80001005120B0349091B09051943114310BD08
:103B9000C40500201F04000010B54C00620D8023F6
:103BA000D218DB00D21A5B057E2A10DD9E3A13DAAA
:103BB000CC170903490819435242D140640001342B
:103BC0001532202A05DAD0400843604310BD00209A
:103BD00010BD0846604310BDC80FC018013810BDA5
:103BE00018B4044B5B6AFC46019308BD24DF7141A5
:103BF00000100000C404002070B513231C78012CB1
:103C000012D0012C12DC214B214A93642148FFF78A
:103C10007BFC214B186070BD1C491D4A98008150E7
:103C200001331F2BF8D9ECE70023FAE71B48FFF715
:103C300073FC05001A48FFF76FFC023803789B00FD
:103C40007F2B09DD12488022290000F00BFC022C9A
:103C500008D0022CDADCD6E7124B134A1348322183
:103C6000FEF7BEFA124B1A88B5231B029A4209D1FD
:103C7000104B1A88104B9A4204D1104B1A88104BE3
:103C80009A42E6D00020FEF743FBC046C53C001038
:103C9000C40400204C330000C4050020534400003D
:103CA00053460000685A00101C5B0010C85A0010F0
:103CB00054380000D8380000494600009C38000005
:103CC0005946000007B56046002800D100BE0188B3
:103CD0000A0A0230DF2AFAD1C9B2820804D3028864
:103CE00040880004104300E00068024A50500390EE
:103CF00007BD0000C40400200FB403BC0CBCF0B529
:103D00000124E407634000E0F0B50C0DCF0F661E00
:103D10003605891B640503D3C943404200D30131F2
:103D2000640D03D0661CF60A07D0E41B00207F0058
:103D3000791C89078912803C24031D0DDF0F6E1E3C
:103D400036059B1B6D0503D3DB43524200D3013381
:103D50006D0D03D06E1CF60A07D0ED1B00227F000C
:103D60007B1C9B079B12803D2D032F1B661B58D489
:103D7000A446202E46DA20371400BC401D00BD406A
:103D8000F24033412A4380185941CB0F05D0C94333
:103D9000C043002264425041514162464D0D28D13A
:103DA0000D0D07D100281FD0241940414941013A87
:103DB0000D0DF9D0640006D3013000D30131002C81
:103DC00001D140084000013A0BD4941CE40A04D10C
:103DD00012051144DB071944F0BDD907204B1943E4
:103DE00000E0D9070020F0BD0029DDD1002CDBD197
:103DF000F0BD0132C6074008CD0728434908002E10
:103E0000E1D0D9E73C2E29DA203E40371400BC40EF
:103E100000D00124F24014431A00BB401C43D317C6
:103E2000ACE7AC46202F08DA20360400B4400D0081
:103E3000B540F84039412843A5E73C2F0CDA203F34
:103E400040360400B44000D00124F8400443080088
:103E5000B1400C43C117EAE710001900002494E7B1
:103E60000000F07FF0B50C0D661E3605891BE60AD2
:103E70006405640D02D0651CED0A04D00020012108
:103E80000905803C2403A4461C0D671E3F05DB1B6F
:103E9000E70A6405640D02D0651CED0A04D0002217
:103EA00001231B05803C24037740644497B484B20B
:103EB00096B27443070C7E43150C6F4380B268437F
:103EC000361802D3012000043F183004350C0019C5
:103ED0007D41844688B29AB250430C0C62431F0C59
:103EE0007C438EB27E43921902D301263604A41974
:103EF0001604170C3618674101BC81B29AB25143BF
:103F0000040C62431B0C5C4380B25843121802D36A
:103F10000120000424181004130C401863412D18CC
:103F20005E410020474106BC88B293B258430C0C56
:103F30006343120C544389B251435B1802D30121ED
:103F40000904641819041A0C091862416D185641C5
:103F50000020474118BCF902720D1143F0026A0DAE
:103F60001043ED020A0D03D16D1940414941013B57
:103F7000124E9B1B7600B3420ED26D0007D3013068
:103F8000002671416646354301D1400840001B05BB
:103F9000C918E4072144F0BD0BDA013306D1013022
:103FA00004D101314F0D01D04908F2E7E1070020AB
:103FB000F0BD013631050020EBE70000FF030000F3
:103FC000F0B51C0D671E3F05DB1BE70A6405640D99
:103FD00002D0661CF60A04D0002201231B05803C97
:103FE0002403D0252D060026F6432E661E096E6694
:103FF000CE0FF619B44649004F0D02D07E1CF60ACA
:1040000003D000200021403F3F033E1BB600B444D4
:10401000013F7F05C91B49082E6F013676089C02B7
:10402000950D25437543ED137543AD1301356D10A3
:10403000F603761B0CB4CC02450D2C43A2B2B3B2EE
:104040005A43270C7B43350C6F43A4B26C431B19B6
:1040500002D3012424043F191C041D0CA4187D4123
:1040600024196D41009A91B2ACB26143170C7C43A4
:104070002B0C5F4392B25A43A41802D301221204BC
:10408000BF182204230C52187B41019C6C431B195E
:10409000520ED9010A434401A01A81B2B2B251436F
:1040A00003145A43360C734387B27743D617D21999
:1040B00000277E4136049B191704160C7F185E41B9
:1040C0007316ED18F301002680337541A90F06D150
:1040D0006400690AE8055B0A184309D22FE004224C
:1040E000944480337541A90AA8059B0A184326D336
:1040F000404149412404009A019B0D005543641B33
:104100004343E41A95B286B27543170C7E43030C01
:104110005F4392B25A43B61802D301221204BF1869
:104120003204330C52197B4152429C41002C02D480
:104130000022013051414008CA071043490802B02B
:104140006246D7079210084BD218084B9A4203D206
:1041500012058918C919F0BD0020002A01DC3900B8
:10416000F0BD01331905F5E7FD030000FE0700006F
:10417000002200B5203200F004F8080000BD000065
:1041800000220B150AD410B5944600F031F814142F
:10419000013400DA0021CB17144C20470020002105
:1041A00070476244343A0CD40C2A07DA0400914078
:1041B000904052422032D440214310BDD843D943CD
:1041C00010BD203207D40C46944052422032114197
:1041D000D040204310BD0800C917203203D45242FA
:1041E0002032104110BD1800190010BDA34100106D
:1041F0000A0DCC0F531E1B05C91A520503D3C94320
:10420000404200D30131520D03D0531CDB0A07D0CA
:10421000121B00206400611C89078912803A120376
:10422000014BD21A70470000FF0300005143434383
:10423000C9188C46110C83B24B4310B4040C614373
:1042400092B280B2504362431C041B0C001910BC94
:1042500059411304120CC0185141614470470000C9
:1042600048404140484000239C46114B5B6818473A
:1042700000239C460E4B1B6818470E4A936F9B0801
:1042800004D200239C460A4BDB681847F0B5146E35
:10429000556E576F166FFFF7F4FF064A14665566A2
:1042A00057671667F0BD00239C46014B9B68184773
:1042B000C8050020000000D0491A002808D108468F
:1042C00070470000C10FC90700D54042002817D031
:1042D000F44603B40B4B1B68984706BC81409E38DC
:1042E0004042803107D20B0607D04900490AC00579
:1042F0001043084360470130F8E7490A8902F5E7AF
:1043000070470000C405002000239C46014B5B6AF7
:1043100018470000C805002070B513231E782A48EE
:10432000FFF7FAF80500012E11D0012E09DDAB1EB2
:104330001B789B007F2B40DD24488022290000F061
:1043400091F82348FFF7E0F8224B186070BD1F4832
:104350005422290000F086F81F4B1A881F4B9A42FE
:104360001CD1A7239B011A881D4B9A4216D11D4BC5
:104370001A881D4B9A4211D11C4B1A8894239B0119
:104380009A420BD11A4B1A881A4B9A4206D11A4BF1
:104390001A681A4B9A4201D1152307E01848FDF715
:1043A000B7FF184C094A99008C5001331F2BF8D9DC
:1043B000144B064A1362D361B7E7134B134A1448F0
:1043C0004221FDF70DFFC04653460000C8050020FE
:1043D0004C330000C4050020EE290000C40F00008B
:1043E000C20D0000962B0000C0B50000182B000085
:1043F000CC2A000010B50000FC2C000051ED8764B1
:10440000A057001015440010305B0010B45B001082
:10441000645B001007B56046002800D100BE01882B
:104420000A0A0230DF2AFAD1C9B2820804D302880C
:1044300040880004104300E00068024A5050039096
:1044400007BD0000C805002001480421014B1847A2
:10445000C002002029350010014B1B6818470000DE
:10446000C0020020014B5B6818470000C00200201A
:1044700010B50300080011001B68984710BD00002C
:10448000F8B507000D001600437D002B02D0002474
:1044900000200CE003681100280098472DE03B7DC8
:1044A00010E03B68154802219847601C0134B44273
:1044B00014DA002CF3DD2B19013B1B780D3B5A421B
:1044C0005341DBB22A5D0A2AF0D1002BEED1A04283
:1044D000E7DA3B68211A28189847E2E7B04203DA86
:1044E0003B68311A28189847002E06DDAD19013DAA
:1044F0002B780D3B5A4253413B75F8BD285C0010A8
:1045000070B505000368002B16D00C4B1C6805E045
:10451000290004C92000FFF7B3FF2469002C09D04B
:104520002368002BF9D0064B1B68002BF0D0A34268
:10453000F3D1EDE700232B6070BDC046AC04002032
:10454000B004002070B505000C000B68802B05D06E
:1045500023685A1C2260E418257170BD0800FFF71B
:10456000CFFFF5E710B5002B02DB0260436010BD02
:10457000024B034A03483F21FDF732FE844D0010F1
:104580002C5C0010A04D001010B582B00400FDF7A7
:1045900073F902000B006846FFF7E4FF009A019BE5
:1045A00022606360200002B010BD000070B582B0D0
:1045B000060014001D00FA22920000230698002134
:1045C000FFF734FE02000B0012196B41002B09DBD0
:1045D0006846FFF7C7FF009A019B326073603000A6
:1045E00002B070BD01225242004BF1E7FFFFFF7F96
:1045F00030B585B004000D0002A8FFF7C5FF029A90
:10460000039B00952000FFF7D1FF200005B030BDCF
:1046100000B583B0FA2189006846FFF7E9FF009AE8
:10462000019B024800F08CFB03B000BDE8020020B3
:1046300010B5024800F06CFB10BDC046E802002037
:10464000F0B5CE46474680B583B006000D009046D3
:104650001C00FFF7DDFF81466B1C05D0002C08D045
:10466000194F1A4B1C6807E0300000F021FB0500D1
:10467000F4E7174FF5E72469002C17D02368002BC7
:10468000F9D0144B1B68002B01D0A342F3D12A00B0
:1046900031002000B8474346002BECD06B46D91DB3
:1046A0000A230B7001222000B847E4E74B46002B99
:1046B00007D16B1E9D41E8B203B0C0BCB946B046FD
:1046C000F0BDFFF7B5FFF4E771440010AC04002023
:1046D00081440010B0040020094A01E010331A00A0
:1046E0001368002B08D08342F8D1002907D1036951
:1046F00013600023036102E0002900D010607047BE
:10470000AC04002010B5064B1C6801E098472469F2
:10471000002C03D06368002BF8D1F8E710BDC04629
:10472000AC04002070B5050000F0C2FA04000023BC
:10473000012201002800FFF783FFFFF7E3FF2000BD
:1047400070BD000070B5A2B004000E00FFF760FF5E
:104750000500002301930A483300220001A9FEF757
:10476000BBFE040001A8FFF7CBFEFFF7CBFF002D37
:1047700002D1200022B070BDFFF75AFFF9E7C04612
:10478000454500100FB400B583B004A901C90191DB
:10479000FFF7D8FF03B008BC04B0184710B500F00D
:1047A000FFF8012010BD000010B582B00C00144BC2
:1047B000C3185A425341134A5B009B5E8B4204D09C
:1047C0006B46DA1D1470002115E06B46DA1D0D23CF
:1047D000137000210029F3D183699B06FCD4137860
:1047E000036001310132F5E783699B06FCD413783D
:1047F0000360013101320029F6D002B010BDC0467D
:104800000080FCBF0007002082B000226B46D91D4B
:1048100006E08369DB06FCD403680B7001320131CA
:10482000002AF6D06B46D87902B0704770B5060002
:104830000D00002405E0315D034B1868FFF7B4FF5D
:104840000134AC42F7DB70BD04070020F8B5060068
:104850000D00002705E07C1CF719FFF7D5FF387025
:104860002700AF4204DA0E4A10688269D206F2D5F8
:104870000C4A1268002A0CD0094A12685021916330
:1048800010003430526B183911408022520102431B
:104890001160002F01D03800F8BD033FFBE7C04690
:1048A000040700203C04002010B5064B1B68002BB9
:1048B00006D0054A126800219163044A106898479F
:1048C00010BDC0463C040020040700204004002026
:1048D00070B505000E001C4B1A681C4BD3185942CA
:1048E0004B4114331C0000281ED0194B1B68002BB1
:1048F00004D0174B1D60174B1E6070BD1649200079
:10490000FCF7FCF801212000FCF7E8F80E4B1B68CF
:1049100050229A63190034315B6B183A1A40802395
:104920005B010B431A60E4E7094B1B68002BE0D0E6
:104930000023936300212000FCF7D0F806492000F3
:10494000FCF706F9D5E7C046040700200080FCBF4D
:104950003C04002040040020A948001070B50D0060
:104960001C000D4B1860002A0BDA002C0EDA0A4BE3
:1049700018682900FDF734FA08480121FFF7ACFE5A
:1049800070BD02211000FBF7A1FFEEE7022120001D
:10499000FBF79CFFEBE7C04604070020D002002095
:1049A00010B5064B1B78064B1B78E1210123002232
:1049B00049020448FFF7D2FF10BDC0464C5D00100D
:1049C000485D00100040034010B504001022002193
:1049D000FFF742FD80235B022360F8235B026360E4
:1049E0008023DB02A360C0231B03A360200010BD53
:1049F0000523CB56002B01DB934211D1094B9C467A
:104A0000604443425841084B8000C0580979012353
:104A10008B40013B9340184043425841C0B270471D
:104A20000020FCE70000D0AF2404002070B50A7914
:104A3000202A19D8174B9C46604443425841164BD4
:104A40008000C45801239340013B497949B20029B1
:104A500010DB08002025AA1A914218DC8B401C426A
:104A600001D00120404270BD0C4B0D4A0D48402141
:104A7000FDF7B6FB2020801A002805DB1A008240D3
:104A80001442F0D00138F7E701204042EBE7012063
:104A90004042E8E70000D0AF24040020845C00100E
:104AA0000C5D0010B05C001070B505000C00160025
:104AB000FFF79EFF002801D0002108E01648FDF70F
:104AC00027FC9A198B1912339B005A510131237913
:104AD0008B4211D9227863781B021343A278120407
:104AE0001A43E3781B0613434A009B5A8022920123
:104AF0009342E6D31A00E5E701229A401300013BF6
:104B0000064A944665446A4255410549AD006A58D3
:104B1000B34013436B5070BDF85C00100000D0AF81
:104B200024040020F8B505000E00FBF7FDFE070089
:104B300031002800FFF77AFF041E09DB0200310074
:104B40002800FFF7B1FF3800FBF7FAFE2000F8BDA0
:104B50000148FDF7DDFBC046F85C0010F0B5C64625
:104B600000B506AC25784C006618F60086193700AB
:104B7000DC373F68BC46CC363668B0466418E40083
:104B8000C83404190434C026B60134438026B60262
:104B90002660002D01D01F2614E0002612E05401EB
:104BA000A0256D0525434C006418E4000419270076
:104BB000DC373D60114D3543D8342560053B053267
:104BC0001F242240052BEAD89B06520113434C00B8
:104BD0006218D20082181500DC352B60074B334376
:104BE000D832136063462B606418E4000019CC309F
:104BF0004346036080BCB846F0BDC04680E000007C
:104C000070B584B004000D00160002680121A940AF
:104C10008A430260002B34D0186869004919C90022
:104C200061180A00C8321060586804321060986831
:104C300004321060DB68DC310B606A005319DB0062
:104C4000D033E318802149010B4380210906196004
:104C50001960164BAB40A3602B1D01210800984042
:104C600080239B012343186028000830814019608D
:104C70001F2333405219D200A418D834236004B043
:104C800070BD6846FFF7A0FE00996B005B19DB0062
:104C9000E3181A00C83211600199043211600299B8
:104CA00004321160039ADC331A60C6E70101010186
:104CB00010B583070AD00300032102E001330B4241
:104CC00005D01A78002AF9D1181A10BD0300196806
:104CD0000C4A0D4C8A188A4322420FD15968094A5E
:104CE00004338A188A43224208D15968054A04339A
:104CF0008A188A432242F1D000E001331A78002A50
:104D0000FBD1E1E7FFFEFEFE80808080F8B5C04663
:104D100001B40248844601BC604700BFC9010020BD
:104D200001B40248844601BC604700BF1502002060
:104D300001B40248844601BC604700BF1502002050
:104D400001B40248844601BC604700BF95010020C1
:104D500053797374656D20636C6F636B206F66208D
:104D60002575206B487A2063616E6E6F74206265D2
:104D70002065786163746C79206163686965766524
:104D80006400000075735F73696E63655F626F6FC7
:104D900074203C3D20494E5436345F4D415800004C
:104DA0002F686F6D652F7370696465725F706967D6
:104DB0002F7372632F632F7069636F2F7069636F36
:104DC0002D73646B2F7372632F636F6D6D6F6E2F16
:104DD0007069636F5F626173652F696E636C756480
:104DE000652F7069636F2F74797065732E6800008A
:104DF00074657374000000007570646174655F759C
:104E0000735F73696E63655F626F6F7400000000AB
:104E100000002050000000001300000012000000FD
:104E2000110000001A00000016000000140000002D
:104E30004001E0013C4E001002FF0000016042B062
:104E4000011401010A1102023A5502003600050060
:104E50002A0000014005002B000001E001021301BF
:104E60000229000030783163203D3D20282A696EF8
:104E70007374293E3E313175000000002F686F6D5C
:104E8000652F7370696465725F7069672F737263F1
:104E90002F632F7069636F2F7069636F2D73646B5D
:104EA0002F7372632F7270325F636F6D6D6F6E2F31
:104EB00068617264776172655F6972712F6972717E
:104EC0002E63000064656C7461203E3D202D3230FD
:104ED00034382026262064656C7461203C3D2032E5
:104EE00030343620262620212864656C7461202603
:104EF00020312900212864656C7461203E3E2031F8
:104F00003175290063757272656E74203D3D205FB6
:104F10005F756E68616E646C65645F757365725F02
:104F2000697271207C7C2063757272656E74203D9D
:104F30003D2068616E646C657200000021657863D5
:104F4000657074696F6E207C7C2065786365707411
:104F5000696F6E203D3D206E756D202B20565441AB
:104F6000424C455F46495253545F4952510000003C
:104F700066616C736500000069735F7368617265D8
:104F8000645F6972715F7261775F68616E646C659E
:104F90007228736C6F745F68616E646C657229004F
:104FA000657863657074696F6E000000666F756E7A
:104FB000640000006972715F6164645F7461696CB0
:104FC0005F746F5F667265655F6C69737400000083
:104FD000696E736572745F6272616E63685F616E41
:104FE000645F6C696E6B00006972715F72656D6FF2
:104FF00076655F68616E646C657200006D616B65FB
:105000005F6272616E6368007265736F6C76655F74
:105010006272616E636800006972715F7365745FCC
:105020006578636C75736976655F68616E646C65DD
:1050300072000000746F74616C0000002F686F6D67
:10504000652F7370696465725F7069672F7372632F
:105050002F632F7069636F2F7069636F2D73646B9B
:105060002F7372632F636F6D6D6F6E2F7069636F37
:105070005F73796E632F6D757465782E6300000021
:105080006D74782D3E636F72652E7370696E5F6C00
:105090006F636B006C6F636B5F69735F6F776E65D7
:1050A000725F69645F76616C6964286D74782D3E07
:1050B0006F776E65722900006D74782D3E656E7491
:1050C00065725F636F756E74000000006D757465C6
:1050D000785F6578697400006D757465785F656EDA
:1050E0007465725F626C6F636B5F756E74696C0080
:1050F0006964202626206964203C3D20706F6F6C17
:105100002D3E686561702D3E6D61785F6E6F6465E0
:10511000730000002F686F6D652F7370696465728E
:105120005F7069672F7372632F632F7069636F2FCE
:105130007069636F2D73646B2F7372632F636F6D70
:105140006D6F6E2F7069636F5F74696D652F746921
:105150006D652E63000000006964202626206964C6
:10516000203C3D20686561702D3E6D61785F6E6FFB
:10517000646573002F686F6D652F73706964657265
:105180005F7069672F7372632F632F7069636F2F6E
:105190007069636F2D73646B2F7372632F636F6D10
:1051A0006D6F6E2F7069636F5F7574696C2F696EB8
:1051B000636C7564652F7069636F2F7574696C2FEC
:1051C00070686561702E6800706172656E745F69E9
:1051D000640000006368696C645F6964000000003B
:1051E000706172656E745F696420213D2063686937
:1051F0006C645F69640000006964000069642026D3
:1052000026202170685F636F6E7461696E735F6ED4
:105210006F646528686561702C206964290000004E
:1052200021686561702D3E667265655F7461696CA9
:105230005F6964002170685F636F6E7461696E738B
:105240005F6E6F646528706F6F6C2D3E686561706E
:105250002C2072657573655F6964290072656D6FD6
:105260007665645F6964203D3D206E6578745F6992
:105270006400000063616C6C6261636B000000009D
:10528000706F6F6C2D3E616C61726D5F696E5F70E7
:10529000726F6772657373203D3D206D616B655F52
:1052A0007075626C69635F69642869645F686967C7
:1052B000682C206E6578745F696429006465666196
:1052C000756C745F616C61726D5F706F6F6C5F693C
:1052D0006E697469616C697A656428290000000050
:1052E000616C61726D5F696420213D20706F6F6C2D
:1052F0002D3E616C61726D5F696E5F70726F677277
:105300006573730072630000417474656D70746539
:105310006420746F20736C65657020696E736964B6
:1053200065206F6620616E20657863657074696FB3
:105330006E2068616E646C65723B207573652062D7
:105340007573795F7761697420696620796F75205C
:105350006D75737400000000616C61726D5F706F39
:105360006F6C5F63616E63656C5F616C61726D0031
:10537000616C61726D5F706F6F6C5F6765745F64A5
:10538000656661756C7400006765745F656E747244
:10539000795F69645F6869676800000070685F66CC
:1053A0007265655F6E6F64650000000070685F6124
:1053B00064645F6368696C645F6E6F6465000000BD
:1053C00070685F696E736572745F6E6F646500000C
:1053D00070685F6765745F6E6F6465006164645FC9
:1053E000616C61726D5F756E6465725F6C6F636B2B
:1053F000000000007570646174655F75735F7369A8
:105400006E63655F626F6F7400000000616C6172B3
:105410006D5F706F6F6C5F616C61726D5F63616C0B
:105420006C6261636B0000006765745F656E747227
:1054300079000000486172647761726520616C6177
:10544000726D20256420616C726561647920636CE3
:1054500061696D656400000074696D65725F6877ED
:105460002D3E696E74732026203175203C3C2061EE
:105470006C61726D5F6E756D000000002F686F6D5E
:10548000652F7370696465725F7069672F737263EB
:105490002F632F7069636F2F7069636F2D73646B57
:1054A0002F7372632F7270325F636F6D6D6F6E2F2B
:1054B00068617264776172655F74696D65722F747B
:1054C000696D65722E630000686172647761726550
:1054D0005F616C61726D5F7365745F746172676543
:1054E00074000000726F6F745F6964002F686F6DE5
:1054F000652F7370696465725F7069672F7372637B
:105500002F632F7069636F2F7069636F2D73646BE6
:105510002F7372632F636F6D6D6F6E2F7069636F82
:105520005F7574696C2F70686561702E6300000090
:105530002170685F6765745F6E6F64652868656178
:10554000702C20726F6F745F6964292D3E736962DD
:105550006C696E67000000002170685F6765745FAA
:105560006E6F646528686561702C20726F6F745F60
:105570006964292D3E706172656E74006E65775F97
:105580007375625F7472656520213D206865617086
:105590002D3E726F6F745F696400000070685F7207
:1055A000656D6F76655F616E645F667265655F6E7F
:1055B0006F64650070685F72656D6F76655F616EC0
:1055C000795F68656164000070685F6164645F634F
:1055D00068696C645F6E6F646500000070685F6787
:1055E00065745F6E6F6465007372635F6672657188
:1055F000203E3D2066726571000000002F686F6DCF
:10560000652F7370696465725F7069672F73726369
:105610002F632F7069636F2F7069636F2D73646BD5
:105620002F7372632F7270325F636F6D6D6F6E2FA9
:1056300068617264776172655F636C6F636B732F0F
:10564000636C6F636B732E6300000000636C6F63A9
:105650006B5F636F6E6669677572650076636F5F17
:1056600066726571203E3D20285049434F5F504C83
:105670004C5F56434F5F4D494E5F465245515F4D1B
:10568000485A202A204D485A292026262076636F22
:105690005F66726571203C3D20285049434F5F5042
:1056A0004C4C5F56434F5F4D41585F465245515FEA
:1056B0004D485A202A204D485A2900002F686F6D06
:1056C000652F7370696465725F7069672F737263A9
:1056D0002F632F7069636F2F7069636F2D73646B15
:1056E0002F7372632F7270325F636F6D6D6F6E2FE9
:1056F00068617264776172655F706C6C2F706C6C3E
:105700002E6300006662646976203E3D20313620BB
:105710002626206662646976203C3D2033323000C4
:1057200028706F73745F64697631203E3D203120AC
:10573000262620706F73745F64697631203C3D20AB
:1057400037292026262028706F73745F64697632AB
:10575000203E3D203120262620706F73745F6469DF
:105760007632203C3D203729000000007265665FDC
:105770006D687A203C3D202876636F5F66726571A4
:10578000202F203136290000706C6C5F696E6974BF
:10579000000000002C2066756E6374696F6E3A20FD
:1057A00000000000617373657274696F6E202225BA
:1057B0007322206661696C65643A2066696C6520B5
:1057C000222573222C206C696E65202564257325A3
:1057D000730A000031203D3D202875696E74707495
:1057E000725F74296C2D3E7370696E5F6C6F636BB2
:1057F000000000002F686F6D652F7370696465721B
:105800005F7069672F7372632F632F7069636F2FE7
:105810007069636F2D73646B2F7372632F727032B4
:105820005F636F6D6D6F6E2F7069636F5F72756E02
:1058300074696D652F72756E74696D652E630000F5
:105840000A2A2A2A2050414E4943202A2A2A0A009D
:105850000A00000072756E74696D655F696E697427
:1058600000000000666E692B00000000666E690093
:105870006E616E00666E692D00000000DE2E001065
:10588000F62E0010F62E0010EA2E0010F62E001054
:10589000F62E0010F62E0010F62E0010F62E001038
:1058A000F62E0010F62E0010D22E0010F62E00104C
:1058B000C62E0010F62E0010F62E0010BA2E001084
:1058C000C62F0010EC2F00100E300010EC2F00102F
:1058D000A62F0010EC2F0010EC2F0010EC2F001062
:1058E000EC2F0010EC2F0010EC2F0010EC2F00100C
:1058F000E22F0010EC2F0010EC2F0010EC2F001006
:10590000EC2F0010EC2F00101A3000107E34001025
:105910009434001094340010943400109434001027
:105920009434001094340010943400109434001017
:105930009434001094340010943400109434001007
:1059400094340010943400109434001094340010F7
:1059500094340010943400109434001094340010E7
:1059600094340010943400109434001094340010D7
:1059700094340010943400109434001094340010C7
:10598000943400109434001094340010C03200108D
:1059900082320010C0320010943400109434001091
:1059A0009434001094340010943400109434001097
:1059B0009434001094340010943400109434001087
:1059C0009434001094340010943400109434001077
:1059D0009434001094340010663000109434001099
:1059E0009434001094340010943400109434001057
:1059F0009434001094340010943400109434001047
:105A0000663000100E33001066300010C0320010F7
:105A100082320010C0320010000000000000F03F91
:105A20000000000000002440000000000000594079
:105A30000000000000408F40000000000088C340CC
:105A400000000000006AF8400000000080842E4141
:105A500000000000D01263410000000084D797418D
:105A60000000000065CDCD412A282875696E743884
:105A70005F74202A29282828766F6964202A2972D1
:105A80006F6D5F646174615F6C6F6F6B75702872AE
:105A90006F6D5F7461626C655F636F646528275327
:105AA000272C202746272929292D322929202A2059
:105AB00034203E3D2053465F5441424C455F5632B0
:105AC0005F53495A450000002F686F6D652F737052
:105AD000696465725F7069672F7372632F632F70DB
:105AE00069636F2F7069636F2D73646B2F737263BB
:105AF0002F7270325F636F6D6D6F6E2F7069636FA1
:105B00005F646F75626C652F646F75626C655F6949
:105B10006E69745F726F6D2E630000005F5F616578
:105B20006162695F646F75626C655F696E6974005C
:105B30002A282875696E74385F74202A2928726FA4
:105B40006D5F7461626C652D322929202A20342012
:105B50003E3D2053465F5441424C455F56325F53B1
:105B6000495A45002F686F6D652F737069646572BF
:105B70005F7069672F7372632F632F7069636F2F74
:105B80007069636F2D73646B2F7372632F72703241
:105B90005F636F6D6D6F6E2F7069636F5F666C6FA3
:105BA00061742F666C6F61745F696E69745F726F88
:105BB0006D2E63005F5F61656162695F666C6F6136
:105BC000745F696E69740000446562756700000067
:105BD000626F6F74325F7732357130383000000099
:105BE000312E352E300000007069636F0000000018
:105BF000636C6163657200004D617920313320323E
:105C00003032330006005250D3F07542C85B0010AA
:105C100006005250E182887FD05B0010060052508F
:105C2000BBFF3CB6E85B00100D0A000075706461B4
:105C300074655F75735F73696E63655F626F6F74C0
:105C4000000000005541525420737464696E0000D6
:105C500055415254207374646F7574005541525409
:105C600020737464696E202F207374646F757400E0
:105C70000600525053B4F4A15C5C0010080052506E
:105C80009200000070726F6772616D2D3E6C656EE0
:105C9000677468203C3D2050494F5F494E53545231
:105CA000554354494F4E5F434F554E54000000003A
:105CB0002F686F6D652F7370696465725F706967B7
:105CC0002F7372632F632F7069636F2F7069636F17
:105CD0002D73646B2F7372632F7270325F636F6DFD
:105CE0006D6F6E2F68617264776172655F70696F46
:105CF0002F70696F2E6300004E6F2070726F677295
:105D0000616D207370616365000000005F70696FF2
:105D10005F66696E645F6F66667365745F666F72F7
:0C5D20005F70726F6772616D0000000020
:105D2C00045C0010105C0010880200101C5C001059
:105D3C0094020010A0020010AC0200107C5C001059
:045D4C00705C001077
:105D500003000068EFF3108C72B60268002AFCD0D2
:105D6000BFF35F8F04229A56002A0BDB002910D064
:105D70000A6000201B68BFF35F8F00221A608CF35B
:105D800010887047D0221206127852B21A71012080
:105D9000F0E70020EEE70000F8B5CE46474680B5B4
:105DA0000400170098460368002B20D0D0231B0660
:105DB0001B785BB299462668EFF3108C72B6356893
:105DC000002DFCD0BFF35F8F04256557002D14DB39
:105DD0002368BFF35F8F00221A608CF310883800AD
:105DE000414600F061F80028E5D000200FE00A4BA2
:105DF0000A4A0B48852100F05FF84B46237123685F
:105E0000BFF35F8F00221A608CF310880120C0BCA2
:105E1000B946B046F8BDC04680500010D8500010BA
:105E20003C50001070B582B0060015001C0001A99E
:105E3000FFF78EFF002807D1019B5BB2D02212062C
:105E4000127852B2934201D102B070BD2A002300F1
:105E50003000FFF7A1FFF7E710B50268EFF31081FC
:105E600072B61368002BFCD0BFF35F8F0423C356B8
:105E7000002B0ADBFF2303710368BFF35F8F00224F
:105E80001A6081F3108840BF10BD034B034A0448D9
:105E9000B42100F011F8C04694500010CC5000100E
:105EA0003C5000107047C04601B40248844601BC13
:105EB000604700BF9117001001B40248844601BC3E
:105EC000604700BFE121001010000000000000004A
:105ED00000000100000000000000000000000200BF
:105EE00000000000000000000000030000000000AF
:105EF000000000000000FF000000000001B548683D
:105F000001318E460047704609380149884701BD76
:105F1000D90C00109C0200200000000008030020A3
:105F20006C04002000000000000000007C04002041
:105F30000000000000000000100000000000000051
:105F4000503300004C330000543300005233000043
:105F50004D5300004D430000533400004334000013
:105F60002D480010000000004D480010D1480010DE
:105F70000000000000010000000000000000000020
:105F800049440010F9340010F93B00101943001087
:045F900031030010C9
:04000005100001E9FD
:00000001FF
